:020000040800F2
:10000000E80700209D010008A50100082122000842
:10001000A9010008AB010008AD01000800000000C4
:10002000000000000000000000000000AF01000818
:10003000B101000800000000B3010008D12F000842
:10004000B7010008B7010008B7010008B7010008B0
:10005000B7010008B7010008B7010008B7010008A0
:10006000B7010008B7010008B7010008C91400086B
:10007000B7010008B7010008F9140008B70100082B
:1000800029150008B7010008B7010008B7010008EA
:10009000CD0C0008B7010008B7010008B70100083F
:1000A000B70100083D300008B7010008B70100089B
:1000B000B7010008B7010008B7010008B701000840
:1000C000B7010008B7010008B7010008B701000830
:1000D000B7010008B7010008F133000841340008F7
:1000E000B7010008B7010008B7010008B701000810
:1000F000B7010008B7010008B7010008B701000800
:10010000B7010008B7010008B7010008B7010008EF
:10011000B7010008A5330008B7010008B7010008BF
:1001200059150008B7010008B7010008B701000819
:10013000B7010008B7010008B7010008B7010008BF
:10014000B7010008B7010008B7010008B7010008AF
:10015000B7010008B7010008B70100089134000892
:10016000B7010008B7010008B7010008B70100088F
:10017000B7010008B7010008B7010008B70100087F
:10018000B7010008B7010008DFF80CD000F0EAFA68
:10019000004800477D380008E807002006488047EF
:1001A00006480047FEE7FEE7FEE7FEE7FEE7FEE75C
:1001B000FEE7FEE7FEE7FEE7E12F00088901000801
:1001C0002DE9FE4F804681EA0300C00F0C460090E7
:1001D00021F0004123F00045B8EB0200A94105D20F
:1001E0004046214690461C460B46024623F00040FE
:1001F000104347D0270DC7F30A00C3F30A510290FA
:10020000401A019040286BDAC3F3130040F4801BBE
:100210000098924620B10023D2EB030A63EB0B0B4C
:1002200001985946C0F14002504600F0D6F9064602
:100230000D4650465946019A00F0EEF910EB0800C1
:100240006141002487EA115284EAE7731A4340D0DF
:10025000009A62B3019A012A4FEA075215DC001B8B
:1002600061EB02014FF0004202EA0752CDE9004281
:10027000001C41F5801132462B4600F025FA03B0F0
:10028000BDE8F08F40462146F9E7001B61EB020113
:10029000001C41F5801300185B412018A2F50017DF
:1002A00047EB030140EAD570B6196D4111E06D08C6
:1002B0004FEA360645EAC0754FEA0752001B61EB6C
:1002C0000201001C41F5801149084FEA3000001975
:1002D000514132462B4603B0BDE8F04F00F0E5B97E
:1002E0000098012240000023D0EB020263EBE07390
:1002F000009821464FEAE074B8EB000061EB04017E
:10030000E9E783F000435BE781F0004158E72DE91E
:10031000FE4F81EA030404F0004421F00041009400
:100320004FF0000B23F0004350EA01045ED052EA84
:1003300003045BD0C3F30A54C1F30A552C44A4F25E
:10034000F3340194A0FB0254C1F3130141F4801172
:10035000C3F3130343F4801301FB024400FB034E79
:10036000840A970A44EA815447EA8357A4FB076842
:1003700002958D0A05FB07854FEA932C04FB0C546C
:100380002705029D4FEA065847EA1637B5EB0805E0
:100390006EEB070C870E920E47EA811742EA831232
:1003A000A7FB0201B6EB0B0164EB00042B0D43EA43
:1003B0000C335E1844EB1C50DA465146E7FB020151
:1003C000C5F313044FEA0B3343EA14534FEA0432E4
:1003D000019C43EA0603A4F10C040294009CCDE9BD
:1003E00000B400F071F903B0BDE8F08F00200146C1
:1003F000F9E72DE9F04D81EA030404F0004B21F008
:10040000004514464FF0000A23F0004150EA05026F
:1004100020D054EA01021DD0C5F30A570246C5F3A5
:100420001303C1F31300C1F30A5640F4801543F4DB
:100430008013A7EB0608101BD64608F2FD3873EBB5
:10044000050002D308F1010801E092185B41B8F100
:10045000000F03DA00200146BDE8F08D00204FF4C4
:100460008011064684460EE0171B73EB050705D383
:10047000121B63EB050306434CEA010C49084FEAE3
:10048000300092185B4150EA0107EDD152EA0300B7
:1004900012D082EA040083EA0501084305D0101B4C
:1004A000AB4106D20122002306E000224FF00043B8
:1004B00002E06FF0010253101AEB06004CEB0851FA
:1004C00010EB0A0041EB0B01BDE8F04D00F0EDB878
:1004D0000EB5C10F80EAE0700844CA07002140F25F
:1004E00033438DE80E000A460B4600F0EDF803B0EA
:1004F00000BD0EB540F2334102910021CDE900115B
:100500000A460B4600F0E0F803B000BD70B5C1F339
:100510000A5201F000450024C1F3130140F2FF33F9
:1005200041F480119A4201DA002070BD40F2334359
:100530009A42A2F2334203DC524200F05DF800E03E
:1005400090402C43F1D0404270BDC1F30A5210B527
:10055000C1F3130140F2FF3341F480119A4201DAF2
:10056000002010BD40F233439A42A2F2334203DC32
:10057000524200F041F810BD904010BD00F0004222
:1005800030F000400AD0C10D01F56071C0F31600D3
:1005900042EA0151C208400711437047002001465A
:1005A000704701F0004330B421F0004150EA0102ED
:1005B00006D00A0DA2F56072C1F31301002A02DC15
:1005C00030BC00207047440F44EAC104C100E01869
:1005D00030BC00EBC25000F031B8202A04DB203AD6
:1005E00000FA02F1002070479140C2F1200320FA86
:1005F00003F3194390407047202A04DB203A21FA84
:1006000002F00021704721FA02F3D040C2F120022B
:100610009140084319467047202A06DBCB17203A41
:1006200041FA02F043EAE07306E041FA02F3D040F7
:10063000C2F1200291400843194670470029A8BF23
:100640007047401C490008BF20F00100704710B4FB
:10065000B0FA80FC00FA0CF050EA010404BF10BCB0
:10066000704749B1CCF1200421FA04F411FA0CF1DD
:1006700018BF012121430843A3EB0C01CB1D4FEA16
:1006800000614FEA102042BF002010BC704700EB11
:10069000C35010440029A4BF10BC7047401C49003F
:1006A00008BF20F0010010BC704710B5141E73F194
:1006B000000408DA401C41F1000192185B411A4322
:1006C00001D120F0010010BD2DE9F04D92469B466E
:1006D00011B1B1FA81F202E0B0FA80F22032904614
:1006E000FFF77BFF04460F4640EA0A0041EA0B0190
:1006F00053465A46084313D0114653EA010019D015
:10070000C8F140025046FFF777FF05460E465046B7
:1007100059464246FFF761FF084305D0012004E037
:1007200020463946BDE8F08D0020054346EAE076D4
:100730002C4337430A986305E40AA0EB0800002223
:10074000FD0A44EA47540A3002D500200146E9E791
:10075000010510196941DDE9084500196941BDE845
:10076000F04DA2E7064C074D06E0E06840F00103BB
:1007700094E8070098471034AC42F6D3FFF708FD21
:10078000D8390008F83900080029816802D041F002
:10079000010101E021F0010181607047084B10B5B3
:1007A000D3F8042307490A40D0E900142143D0E9D3
:1007B0000240044321431143C3F8041310BD000059
:1007C00000200140E030FCFF1FB51FA04FF4C662BF
:1007D000006803901D49202000F0E5F81C4C04221D
:1007E0002146104600F0DFF808222146042000F0E0
:1007F000DAF810222146042000F0D5F8154901222C
:10080000881500F05BF90220134C009003AB2246E0
:100810004FF02061400200F07FF80022114638209E
:1008200000F004F90D4B22469905081100F034F848
:100830000B4A0C4908208DE807000B4B142253216A
:100840000A4800F06DF91FBD0C0D000000140240B5
:1008500000080240002001400022014010640240D4
:10086000793200081932000869250008000C0040A0
:100870000029816802D041F4807101E021F4807187
:10088000816070470029816802D041F4007101E065
:1008900021F400718160704770B50D4690B01E461E
:1008A0001446012101F054FE1A480021CDE902014D
:1008B0000220CDE90401400206904000079080002C
:1008C00008904011CDE909010120CDE90B104C340D
:1008D000CDE900540D910E916946304600F0CEFFEF
:1008E0000C490022091D304600F06EFF0121304600
:1008F00000F060FF1021304600F0AAFE0122102116
:10090000304600F0A5FF0121304600F0B7FE10B0E0
:1009100070BD0000640000202DE9F0418AB00F4650
:100920001E46904604460121109D01F029FE01213A
:10093000204601F031FE0021204601F02DFE00246A
:1009400006944FF480300994CDE9070406A8FFF718
:1009500025FF01208DF804000007CDE9020700946F
:100960008DF8054004948DF814506946404600F017
:1009700037F807E0601CC2B2315D0623404600F044
:1009800063F8641CAC42F5DB01214046FFF77AFFB7
:1009900001214046FFF76CFF01214046FFF7F4FEBE
:1009A0000AB0BDE8F0817CB50D461446012101F086
:1009B000CFFD03228DF80420002200948DF807203B
:1009C0006946284601F05EFA7CBDC06C80B2704773
:1009D0000246002012680A4200D001207047000041
:1009E00030B542680F4B0C791A400B6842EA04227A
:1009F0001343436082680C4B4D791A40D1E903439D
:100A000023438C6844EA4504234313438360C26A4A
:100A1000097D22F47002491EC9B242EA0151C16245
:100A200030BD0000FFFEFFFCFDF7FFC008B58DF8EC
:100A300000008DF801108DF8022001208DF80300D0
:100A4000684601F00FFD08BD70B5072609290AD9CF
:100A5000C568A1F10A0404EB4404A640B543A340D1
:100A60001D43C56007E0056901EB4104A640B5439D
:100A7000A3401D4305611F23072A09D2446B521E60
:100A800002EB820293409C4391400C43446370BD4F
:100A90000D2A09D2046BD21F02EB820293409C43C1
:100AA00091400C43046370BDC46A0D3A02EB8202AC
:100AB00093409C4391400C43C46270BD70B50E4698
:100AC0008AB015460446012101F05AFD0121204655
:100AD00001F062FD0021204601F05EFD0024069435
:100AE0004FF480300994CDE9070406A8FFF756FEBD
:100AF00000948DF804408DF80540029404948DF81C
:100B0000145069463046FFF76BFF01213046FFF76E
:100B10003BFE0AB070BD816841F080418160704742
:100B20002DE9F04188B08046DDE90E060F461446F7
:100B30000121109D98470020ADF80070ADF8080025
:100B4000ADF802008DF80A0001946946404602F0B3
:100B5000EBFB0A2005906020ADF80C000120ADF8F9
:100B60000E000220ADF8180003A94046B047082146
:100B70004046A8470121404602F0F1FA30214046A4
:100B800002F0CAFB0121404602F0DFFA08B0BDE8DE
:100B9000F08100001E4800B59FED1C0A012180ED88
:100BA000000A9FED1C0A80ED010A9FED1B0A80EDF3
:100BB000020A0C30B2EE0E0A80ED010A9FED170A10
:100BC00080ED000AB0EE040A80ED030AB0EE0C0AD4
:100BD00080ED020A9FED120A80ED040AA0F53B7039
:100BE00002F0C0F802210F4802F0BCF80D480921BC
:100BF000B83002F0B7F806480A21B83802F0B2F867
:100C0000094801218164C16400BD00009A99193F1F
:100C1000B00300209A99993E00000000000096431E
:100C200000008C42880100200000002010B504461E
:100C300090F876000A283FD1092104F16C0002F0F7
:100C40000DFE94F87510884236D194F86C00DFEDF3
:100C50001C0A00EE100AB8EE400A84ED1F0AB4F830
:100C60006D0040BA00EE100AB8EE400A80EE201A7D
:100C700084ED201AB4F8710040BA00EE100AB8EE04
:100C8000400A84ED210AB4F8730040BAA4F8780051
:100C90002178092901D00A290BD1FFF72AFC9FED01
:100CA000091B53EC112BFFF732FBFFF74EFCA4F8A6
:100CB0007800204600F044FF002084F8760010BD44
:100CC0000000C8422DB29DEFA7C6E73F2DE9FE4FB9
:100CD0000026344602A96846029600F041F98B4A84
:100CE0000299DFF82CB2914261D19DF80100FF28F2
:100CF00011D0F02859D19DF80000864D864C0F2860
:100D00004FD2DFE800F04E0B11174E4E4E1D232937
:100D10002F353B3E46000D20804945E0684601F0F6
:100D200093FC85ED000A3CE0684601F08DFC85ED02
:100D3000010A36E0684601F087FC85ED020A30E0E2
:100D4000684601F081FC84ED030A2AE0684601F060
:100D50007BFC84ED020A24E0684601F075FC84ED1A
:100D6000040A1EE0684601F06FFC84ED010A18E0F9
:100D7000684601F069FC84ED000A12E002F00EF80A
:100D80000FE0684601F060FCBDEEC00A8BED000A82
:100D900007E0684601F058FCBDEEC00A604880EDEF
:100DA000000A9DF800005F490870BDE8FE8F5E4AAA
:100DB0009142FAD10DEB00085C4D18F8011CDFF8E8
:100DC00070915C4B6A46CF0906D01E7089F80060AE
:100DD00001F01F0702242F7095F800C001F01F07D3
:100DE000554D674526D1C1F3401C99F800108C453C
:100DF00020D139B1002189F80010504F9246A0F15E
:100E0000010C15E00121F6E719787A68914200DDBE
:100E100079600C2905D908F8016C1E7089F800600A
:100E200008E01AF804206A54491C641C1970E4B2E2
:100E30006445E9DB18F8011C4906B6D50828B4D189
:100E4000187898460C285CD101F006FADBF800000F
:100E50000028A88800D0404201B2394890F8A80084
:100E600010B9374801F05CFC2D4800680028E8887C
:100E700000D0404201B2334890F8A80010B9314880
:100E800001F04EFC68884FF4FA6701B201F57A7000
:100E9000B8420DD82C4C94F8A80048B9204601F06F
:100EA0003FFC94F98910B4F9040001F047F8E0839D
:100EB000288801B201F57A70B8420DD8234C94F815
:100EC000A80048B9204601F02BFC94F98910B4F928
:100ED000040001F033F8E0831D4C1E4F2889208068
:100EE000387858B14FF400711B4801F017F828B159
:100EF000208818B93878401E3870268017496889CC
:100F0000088088F8006089F800604EE70A574E01B3
:100F100048000020B0030020BC0300200200002095
:100F20004C000020010000200A554E01AE000020B8
:100F3000AD000020AC000020D0030020B000002055
:100F400040020020F8020020D0000020880100208C
:100F50000800002003000020000402400A000020D6
:100F600070B50F4E0D46044686B00021304600F0A5
:100F700074F9002812D06A460021304600F0D5F9F5
:100F8000019828600021684603E04218D27A625432
:100F9000491C9DF80A208A42F7D8D0B206B070BD2D
:100FA00000640040F0B585B00023CDE90031042194
:100FB0008DF808108DF809308DF80A20694604E094
:100FC000C45CCD185B1CEC729BB29342F8D30C4FFF
:100FD000384600F0F1F90646002440F6FF7501E0BE
:100FE000641CA4B23146384600F038FA08B9AC4265
:100FF000F6D3AC4202D3012005B0F0BD0020FBE7E0
:101000000064004038B50F4D09240B234FF40062F3
:1010100029460120009400F083F80C23AA142946E5
:101020000120009400F07CF801220621142000F039
:101030006EF901B02802BDE83040034B034A044971
:1010400000F016B9000002400A574E010A554E0141
:1010500000640040F0B5827A2F4D012191402A684A
:1010600042F001022A602C4E1C3632688A433260FC
:10107000294A047B294B0C32A4B914688C431460B0
:101080004488C78844EA0744877A03EBC707C7F850
:1010900040460488878844EA0744877A03EBC707F9
:1010A000C7F84446047B012C12D114680C43146029
:1010B000847A026803EBC4044FEA3242C4F8402643
:1010C000847A426803EBC4034FEA3242C3F84426F1
:1010D000114AC37A121D002B136806D00B4313600C
:1010E0000D4A0389143213B104E08B43F7E7136808
:1010F0008B4313600389012B02D113680B431360E8
:10110000407B012802D1306808433060286820F015
:1011100001002860F0BD0000006600400060004053
:101120002DE9FC410D461F4614460121089E01F0A1
:101130000FFA32463946284600F0E0FE02218DF8CB
:10114000041000218DF8061003208DF80500012001
:101150008DF8070000946946284600F093FEBDE82C
:10116000FC81002A426901D00A4300E08A434261BF
:10117000704710B50368002223F002030360036880
:1011800043F0010303604FF6FF7300E0521C446814
:10119000E40701D19A42F9D14268D2073ED08A7958
:1011A000012A02683CD022F080020260CA79012A3A
:1011B000026838D022F0400202600A7A012A0268EE
:1011C00034D022F0200202604A7A012A026830D02C
:1011D00022F0100202608A7A012A02682CD022F0E2
:1011E00008020260CA7A012A026828D022F00402AA
:1011F00002608A78CC78920742EA04620C7942EA6B
:1012000004424C79098842EA0452491E0A43C261E9
:10121000016821F001010160002114E0002010BDEF
:1012200042F08002C1E742F04002C5E742F02002EE
:10123000C9E742F01002CDE742F00802D1E742F0E0
:101240000402D5E7491C4268D20701D09942F9D17E
:101250004068C007E2D1012010BD0246002029B13C
:10126000012902D1106900F003007047D068FAE745
:101270002DE9F041884688B01E461746012101F04D
:1012800073F900248DF806408DF8074007208DF88B
:10129000040004208DF8084001258DF802408DF8E7
:1012A00005008DF809508DF8034006208DF80A409E
:1012B000ADF800008DF80B4069464046FFF759FF36
:1012C000780BADF80C004FF6FF7000EAC701091D5E
:1012D000ADF80E10710B00EAC6008DF81640ADF89F
:1012E0001010001D8DF817508DF81850ADF8120031
:1012F000ADF814408DF8195003A8FFF7ABFE01229A
:1013000002214046FFF72DFF08B0BDE8F08108B587
:101310008DF800008DF801108DF8022001208DF865
:101320000300684601F09EF808BD10B500EB0113FC
:10133000D3F8B04114F004041472D3F8B04133D0A0
:10134000E4085460D3F8B04104F002045472D3F8B6
:10135000B44104F00F049472D3F8B441240AD47455
:10136000D3F8B841D472D3F8B841240A1473D3F82F
:10137000B841240C5473D3F8B841240E9473D3F8B5
:10138000BC41D473D3F8BC41240A1474D3F8BC41D3
:10139000240C5474D3F8BC311B0E937439B1016919
:1013A00041F02001016110BD640D1460CAE7C168FD
:1013B00041F02001C16010BD30B5024600209368A5
:1013C0005B0108D49068000101D5012003E090681A
:1013D000C00037D5022002EB0012D2F8803103F0B2
:1013E0000103C2F880310B7A73B3D2F880414D68A3
:1013F0001C434B7A43EAC5031C43C2F880418B7AF5
:1014000003F00F038B72D2F8843123F00F03C2F87C
:101410008431D2F884318C7A2343C2F88431CB7A78
:10142000CC6843EA0423C2F88831CB7B096943EADC
:101430000121C2F88C11D2F8801141F00101C2F8EB
:10144000801130BD042030BDD2F880314C7A234366
:101450000C8843EA4453C2F88031D0E7002221B11E
:10146000012905D0022906D112E08268114801E065
:101470008268114802401149501A8A4214D00ADC8D
:10148000A2B16FF0806010180FD002280CD10FE0CD
:1014900082680B48EEE7B0F5007F09D00949401893
:1014A00003D0B0F5003F03D0002070470220704702
:1014B0000120704703000004000300080001000839
:1014C000000003100001FFF770B5094D094C2946D3
:1014D000204600F093F9002809D02946204600F064
:1014E000B7F82046BDE87040002100F0C7B870BDD5
:1014F000208000101060024070B5094D094C29464B
:10150000204600F07BF9002809D02946204600F04B
:101510009FF82046BDE87040002100F0AFB870BDD4
:10152000008000185860024070B5094D094C2946EA
:10153000204600F063F9002809D02946204600F033
:1015400087F82046BDE87040002100F097B870BDD4
:1015500000880020886002402DE9F0412D4D2E4C7E
:101560002946204600F04AF900284ED02946204658
:1015700000F06EF8204600F039F9284AF0B3284808
:10158000284BDFF8A4C0018811804088508058881B
:10159000264E401C81B259801088DCF800404FF480
:1015A000C8772044CCF8000052883468151935609B
:1015B000B9422AD300EE100A1D4A0121B8EE400AB2
:1015C000117000245C80E04610EE100AFEF7D6FF92
:1015D0009FED181B53EC112BFEF799FE9FED171B87
:1015E00053EC112BFEF705FFFEF7DBFF15490860F2
:1015F000B5FBF7F080B2C8F8004000E007E000F06B
:10160000FFFC114880ED000A3460BDE8F0810F480E
:10161000B6E700002080001010640240DC030020C8
:1016200068000020B000002058000020B800002012
:101630000500002043CA4FAA7D3A0A40000000007E
:101640000000F940540000205000002064000020F9
:10165000074A904201D2074801E005481038064A7F
:101660008B0001EA020101D5C160704781607047BB
:1016700010640240006002407D0F7D0F0029016868
:1016800002D041F0010101E021F001010160704749
:101690002DE9F043016821F00101016000210160A2
:1016A00041608160C1600161212141613C493C4A46
:1016B0003D251039904202D18D60BDE8F083384A53
:1016C0004FF474661832904201D18E60F5E7344AC7
:1016D0004FF474173032904201D18F60EDE7304AF9
:1016E0004FF0746C4832904202D1C1F808C0E4E770
:1016F0002B4B2C4A6033984201D1CA60DDE7284C5D
:10170000294B7834A04201D1CB60D6E7DFF8908036
:10171000264C08F19008404501D1CC60CDE7DFF8B8
:1017200080804FF03D5908F1A808404502D1C1F82A
:101730000C90C2E71E49DFF878800839404501D196
:101740000D60BAE71A4D1835A84201D10E60B4E712
:10175000174D3035A84201D10F60AEE7144D483522
:10176000A84202D1C1F800C0A7E7114D1049603569
:10177000091FA84201D10A609FE70D4A78329042C2
:1017800001D10B6099E70A4A9032904201D10C6076
:1017900093E7074AA83290428FD1C1F800908CE7B6
:1017A000106002403D000020400F002000003D205E
:1017B000106402400029016802D041F4802101E058
:1017C00021F4802101607047002A026802D042F4AF
:1017D000002201E022F4002202600161704701460C
:1017E00000200968C90700D0012070470146002089
:1017F0000968090300D501207047000030B5104A80
:101800000024904201D20F4A01E00D4A103A0E4BDB
:10181000194205D01E2303EAD12503682B4002E0BC
:10182000406900F08003880001D5506800E010682E
:10183000064A1040084201D003B10124204630BDC1
:1018400010640240006002403C0F3C0F7D0F7D0F92
:101850000B0607D5436912B143F0800301E023F082
:1018600080034361802908D0002A026801F01E012C
:1018700001D00A4300E08A430260704730B5036834
:10188000124ACC6813400A682243D1E905452C432B
:101890002243CC6922430C6A22434C6A22438C6A5D
:1018A00022434C6B22438C6B22431A4302604269F1
:1018B00022F00703D1E90B2422431A4342610A694B
:1018C00042604A6882608968C16030BD3F801CF018
:1018D0002DE9F0438FB08846DDE916658146012188
:1018E0001C461746480500F033FE3846FFF7D0FE89
:1018F0003846FFF774FF0028FAD14020CDE90250A6
:101900001220049000204FF48061CDE90501890088
:1019100007918900CDE908108900CDE90A1003215B
:10192000CDE90C10CDE900460E9069463846FFF728
:10193000A5FF01224146484601F01CFC1021384613
:10194000FFF786FE012210213846FFF781FF0021B4
:101950003846FFF793FE0FB0BDE8F0832DE9FE4F48
:1019600001263A4F0523202239463046009600F0E2
:1019700083F8DFF8E0A04524CDE9004ADFF8D08005
:101980000323A20701213448CDF8088000F0A3F812
:1019900000221146102000F090F802250723802233
:1019A00039460120009500F067F8DFF8B0902C4F21
:1019B0008DE8900203232B4A0221274800F08BF880
:1019C00000221146102000F078F8DFF89CB00723C1
:1019D000802259460220009500F04EF88DE89002D2
:1019E000224F03233A4604211B4800F074F80022DA
:1019F00011460E2000F061F80623402259460220CD
:101A0000009500F039F8CDE9004A03233A46042155
:101A10001148CDF8088000F05EF8002211460B2036
:101A200000F04BF840F28F11CDE900160020029033
:101A300053230F4A01210F4801F0B8FB03B00022E5
:101A4000BDE8F04F0121192001F0D7BB0000024092
:101A500079320008193200086925000805330008AA
:101A600085320008000400400004024000080040E5
:101A700000000140812500082DE9FC410D461F466C
:101A800014460121089E00F063FD3246394628467F
:101A900000F034FA02218DF8041003218DF80510AE
:101AA00000208DF8060001208DF80700009469469B
:101AB000284600F0E7F9BDE8FC8108B58DF8000084
:101AC0008DF801108DF8022001208DF80300684682
:101AD00000F0C8FC08BD2DE9F041904688B00246F0
:101AE0000EA81C4690E8E0000B46012118469047DE
:101AF000ADF800400024ADF80840ADF80240019573
:101B00008DF80A406946404601F00EFC6020ADF8B1
:101B10000C000120ADF80E000594ADF8184003A9A3
:101B20004046B04708214046B8470121404601F0F1
:101B3000FFFA0121404601F008FB08B0BDE8F08142
:101B4000B0F878100D4A00EE101AD2ED070AB8EE80
:101B5000400A92ED081A41EE000A00EE101A92EDCA
:101B6000091AB8EE400A20EE011A00EE101AB8EE7B
:101B7000400A41EE000AC0ED250A7047000000202F
:101B800005490028086802D040F4806001E020F494
:101B90008060086070470000003C024070B5064657
:101BA000002529B1012927D0022928D04FF44075FA
:101BB00000F080F809281ED1124C206820F44070F3
:101BC0002060206828432060206820F0F800206012
:101BD000206846F0020108432060206840F480300D
:101BE000206000F067F8216821F00201216021687F
:101BF00021F0F801216070BD4FF48075D8E74FF4F3
:101C00000075D5E7103C02400D4909200A68D2034F
:101C100001D5012070470A68D20601D50620704719
:101C20000A68D20501D5022070470A6812F0E00F59
:101C300001D00720704709688907FBD50820704745
:101C40000C3C02400248016841F0004101607047CD
:101C5000103C024070B50D46064600F02BF80928EE
:101C600013D10A4C206820F440702060206840F4B2
:101C700000702060206840F001002060356000F0B6
:101C800019F8216821F00101216070BD103C02406B
:101C900005480068002805DA034804490C3801604B
:101CA0000349016070470000103C02402301674572
:101CB000AB89EFCD08B509208DF80000FFF7A4FF30
:101CC0008DF800009DF800000128F7D09DF8000075
:101CD00008BD000010B5234800F07EFD224988426F
:101CE00001D000F047F81F48001D00F0A9FC1F4C70
:101CF0001C4884ED000A083000F0A2FC194884ED6D
:101D0000010A0C3000F09CFC164884ED020A2030D9
:101D100000F096FC0C34134884ED030A1C3000F0EC
:101D20008FFC104884ED020A243000F089FC0D4835
:101D300084ED040A283000F083FC0A4884ED010A8F
:101D40002C3000F07DFC074884ED000A303000F0B4
:101D500043FD074CA0640348343000F03DFDE064CF
:101D600010BD00000000060878563412B0030020B1
:101D70000000002010B572B601222949294800F060
:101D80002DFD00F069FA274801222749001D00F0C7
:101D900025FD254923480122091D083000F01EFDBC
:101DA00021492048012208310C3000F017FD00F0D5
:101DB00053FA1D491B4801221831203000F00EFD56
:101DC00019491848012214311C3000F007FD16494A
:101DD000144801221C31243000F000FD00F03CFAD0
:101DE0001149104801221031283000F0F7FC0E494B
:101DF0000C4801220C312C3000F0F0FC00F02CFAE1
:101E0000084801220949303000F0E8FC074905483C
:101E10000122091D343000F0E1FC62B610BD000063
:101E20006C00002000000608B003002048000020DD
:101E30007CB50D461446012100F08AFB01228DF885
:101E4000042000208DF8060003208DF80500009482
:101E50008DF807206946284600F014F87CBD7CB553
:101E60000D461446012100F073FB00228DF804207A
:101E70008DF8062000948DF807206946284600F06A
:101E800001F87CBDF0B5002201274FF0030C0B6870
:101E900007FA02F52B40AB422CD1066853000CFA2E
:101EA00003F4A64306600E79D0F800E09E4046EAAF
:101EB0000E0606600E79012E01D0022E12D1866820
:101EC000A64386604E79D0F808E09E4046EA0E06AA
:101ED00086604668AE43466045688E799640B6B2E5
:101EE00035434560C568A543C560CC799C40C3684F
:101EF0001C43C460521C102AC9D3F0BD4B07DB0E33
:101F00009A40C90810B500EB8100016A0F249C407B
:101F1000A1430162016A1143016210BD0246002023
:101F200012690A4200D00120704741837047018343
:101F3000704742694A4042617047000070B50C46E4
:101F4000054610FB04F0FEF7C3FA41EC100B002D20
:101F50000DDB51EC100B9FED121B53EC112BFEF718
:101F6000D6F9FEF7D3FA80B240F2AE3110E09FED21
:101F70000E1B51EC100B53EC112BFEF7C8F9FEF7BA
:101F8000C5FA0B4901FA80F0404280B240F26C7110
:101F9000884200D90846002C00D1002070BD000006
:101FA000AF25E4839ECDBA3F9A9999999999B93F03
:101FB000E9FBFFFF10B50C4601F0F4FBC1B294F849
:101FC00076000A2802D204F16C02815414F8760FCC
:101FD000401C207010BD10B5044607230122FEF7F7
:101FE00033FD2046FEF797FD02212046FEF7F0FC68
:101FF0000028F9D02046BDE81040FEF7E6BC0000FE
:1020000010B52DED068BDFED5E8A9FED5E8AFEF743
:1020100070FA9FED5D9B53EC192BFEF778F99FED5D
:102020005C1B53EC112BFEF7E4F9FEF7BAFA0AEE4B
:10203000100A1AEE100AFEF7A1FA53EC192BFEF75C
:1020400063F928EE8A0A41EC190B10EE100AFEF72C
:1020500095FA53EC192BFEF7CCF9FEF7A2FA4E498C
:1020600088427DDC4D499FED4E8B884210DDFEF7A6
:1020700085FA9FED4D1B53EC112BFEF748F953ECFD
:10208000182BFEF7B6F941EC100B9FED491B62E0EF
:102090004949884210DDFEF771FA9FED481B53EC69
:1020A000112BFEF734F953EC182BFEF7A2F941EC93
:1020B000100B9FED441B4EE04449884210DDFEF7B3
:1020C0005DFA9FED431B53EC112BFEF720F953EC07
:1020D000182BFEF78EF941EC100B9FED3F1B3AE0F9
:1020E0003F49884210DDFEF749FA9FED3E1B53EC55
:1020F000112BFEF70CF953EC182BFEF77AF941EC93
:10210000100B9FED3A1B26E03A49884210DDFEF79E
:1021100035FA9FED391B53EC112BFEF7F8F853EC11
:10212000182BFEF766F941EC100B9FED351B12E002
:10213000354988421CDDFEF721FA9FED341B53EC34
:10214000112BFEF7E4F853EC182BFEF752F941EC93
:10215000100B9FED301B51EC100B53EC112B00E0DA
:1021600008E0FEF72DF8FEF71CFA08EE100A01E071
:102170009FED2A8AB0EE480ABDEC068B10BD000028
:1021800000401C46000000006666666666660A40FF
:102190000000000000FEAF4000E8FA4600907446E0
:1021A0000000000000408F40A245B6F3FDD4ECBF14
:1021B000A8C64B3789613C4000D8CB45DFE00B9384
:1021C000A90204C06ABC7493185449400080394580
:1021D000F54A5986385619C0A245B6F3FD4C52400F
:1021E000008099448D976E12830030C0BE9F1A2FD5
:1021F000DDA45840004024444A0C022B874643C0CB
:1022000085EB51B81E355F400000A2438716D9CE3A
:10221000F77354C03D0AD7A370D562400000FA425C
:10222000FEE770B504460D4645F2555000F02AF819
:10223000204600F01BF8284600F01EF800F00EF8CB
:10224000BDE87040AFF3008002494CF6CC40086016
:102250007047000000300040AFF3008002494AF6AA
:10226000AA20086070470000003000400149486023
:10227000704700000030004001498860704700004E
:102280000030004001490860704700000030004005
:10229000012202492020FFF7CBBD000000140240BC
:1022A00010B50C494FF0E02348689A694C68A04289
:1022B000FAD1096801EB4103C3EBC113C2EBC302BE
:1022C000B2FBF1F100EB4002C2EBC01001EBC00029
:1022D00010BD00005C00002030B5B0F90430002AC9
:1022E00075D0B0F97820C280048913FB04F500246E
:1022F0009FED581A002D08DA002A06DD848080ED53
:10230000031A80ED041A048104E00381002B01DD2F
:102310009A1A02E0B0F904301A4400EE102AB8EE1E
:10232000C00A80ED030AD0ED040A91ED002A828BE9
:1023300070EE601A61EE821A91ED012A42EE001AE7
:10234000B0EE002A00EEC20AD0ED050A30EE200AF7
:10235000D1ED020A40EE801ABDEEE10A10EE101A2D
:10236000114409B28183B0F90420002A03DB00295B
:1023700003DC002101E00029FBDA13328183272AE4
:1023800007D2848380ED031A80ED041A80ED051ACC
:1023900005E0B0F91C2040F217418A4201DAB0F999
:1023A0001C102D4A8183914200DC11468183002953
:1023B00002DAA1F217414942C18390ED040A80ED8F
:1023C000050A90ED030A80ED040A30BDFFE7B0F87E
:1023D000781042F21072002B1ADB40F6057461434C
:1023E0001E4C2144B1FBF2F189B240F252329142CB
:1023F00003D84FF4A072914200D2114603EB43027E
:102400009200A0F8681012B2C28320E0C183DCE71A
:1024100001EB4114C4EB4121114C04EBC101B1FBB0
:10242000F2F189B24FF44872914203D84FF48C72A2
:10243000914200D21146A3EB83024FF48363A0F8CC
:10244000681003EB820212B2C28301F583618A42F3
:10245000DCDABAE70000000018FCFFFFC07D1C00BA
:102460004005150030B50F23C27801780125FAB177
:10247000144A126801F1E02102F4E062C2F5E06260
:10248000C2F30722C2F10404D3404278A240847808
:102490001C401443220181F80024007800F01F0141
:1024A0008D404009800000F1E020C0F8005130BDAF
:1024B00001F01F0085404809800000F1E020C0F8CD
:1024C000805130BD0CED00E002490843024908602C
:1024D000704700000000FA050CED00E0034840786A
:1024E000002801D000F092BB7047000000000020DF
:1024F00070B5144C042221460120FFF7B0FC4FF4C4
:10250000407211490220FFF7AAFC48F2020221465C
:102510000120FFF78DFC0D4E4FF400452A46314651
:102520002020FFF785FC02212046FFF700FD294609
:102530002046FFF7FAFC29463046BDE87040FFF719
:10254000F4BC0000000002400004024000140240FD
:10255000044A0029116801D0014300E08143116061
:102560007047000030380240044A0029116801D049
:10257000014300E081431160704700004038024091
:10258000044A0029116801D0014300E08143116031
:102590007047000044380240044A0029116801D005
:1025A000014300E08143116070470000243802407D
:1025B00070B5204B1968204C11F00C0104D0661046
:1025C000042903D0082903D004601BE0066019E049
:1025D000184A121F1168C1F38055116801F03F01BC
:1025E00015B1B6FBF1F101E0B4FBF1F1146812682A
:1025F000C4F388146143C2F30142521C5200B1FB80
:10260000F2F1016019680F2202EA11110B4A545CC1
:102610000168E14041601C68072505EA9424145DC7
:1026200021FA04F484601B6805EA5333D25CD1407C
:10263000C16070BD083802400024F400BC000020D6
:1026400090ED000A7047000070B504462DED048B34
:10265000857905F00F00FDF74CFF9FED2C1B53EC27
:10266000112BFDF754FE41EC180B2809FDF741FF33
:102670009FED281B53EC112BFDF749FE41EC190B84
:10268000A078264A0109514300F00F0043F6095291
:1026900010FB02F001EB8011E07840F635430209AF
:1026A00012FB03F201EB421100F00F0040F2712225
:1026B00010FB02F001EB00122179080900EB400346
:1026C000C3EBC01002EBC00201F00F0000EBC00131
:1026D00001EB001002EB80026079010901EB81013E
:1026E00002EB410100F00F000844FDF7F1FE53EC4E
:1026F000192BFDF765FD53EC182BFDF761FDFDF778
:1027000050FFBDEC048B00EE100A70BD7B14AE4789
:10271000E17A843F9A9999999999B93F809698005E
:10272000B0F90820002A03DA002901DB8188891C1E
:1027300081800181704700001C49884201D200203D
:1027400070471B49884201D20820704719498842C6
:1027500001D2102070471849884201D218207047D2
:102760001649884201D2202070471549884201D27B
:10277000282070471349884201D2302070471249FF
:10278000884201D2382070471049884201D2402047
:1027900070470F49884201D2482070470D4988424E
:1027A00001D25020704758207047000000400008B8
:1027B0000080000800C000080000010800000208B6
:1027C00000000408000006080000080800000A08CD
:1027D00000000C0800000E08006870472DE9F04169
:1027E00004461D48092690460F46844231D3A0076F
:1027F0002FD1FFF74DFA0020FFF7C2F91748254601
:1028000004EB880884420ED31AE02868401C09D0E3
:102810002846FFF791FF0221FFF7C0F90646092875
:1028200001D00FE02D1D4545EFD3092E08D009E05A
:1028300020463968FFF70EFA092803D1241D3F1DF1
:102840004445F5D30120FFF79BF9BDE8F041FFF7C0
:10285000F9B9BDE8F0810000000006080000FF1F84
:10286000174A30B4174832F8781FA0F10C030170F2
:1028700092F91120090AC2F10A0241EA0211124A30
:10288000417032F8781F817092F91120090AC2F163
:102890000A0241EA0211C170002202714271827182
:1028A000D97801F1C004C471491CC8B2D87020287D
:1028B00000D3DA7030BC082204490248FEF772BB2C
:1028C000880100207C000020D000002001534E1F12
:1028D000114A124891880170090A4170104989888B
:1028E0008170090AC170D18B0171090A41710321FC
:1028F000A0F114028171D17801F1C003C371491CA8
:10290000C8B2D070202801D30020D0700822054919
:102910000248FEF747BB0000D000002084000020E2
:102920008801002001534E1F144830B4C18B144855
:102930000022144B0170090A41708270C27033F892
:10294000781F017193F91130090AC3F10A0341EAB2
:10295000031141710621A0F11C048171E17801F19C
:10296000C003C371491CC8B2E070202800D3E270D4
:1029700030BC082204490248FEF714BB880100203D
:102980008C0000204002002001534E1F134A30B437
:10299000134832F8781FA0F12403017092F9112036
:1029A000090AC2F10A0241EA021141700022827052
:1029B000C2700271427109218171D97801F1C0049C
:1029C000C471491CC8B2D870202800D3DA7030BC5A
:1029D000082204490248FEF7E5BA0000F802002088
:1029E0009400002001534E1F1B48F2EE040A90EDA4
:1029F000000A1A4820EE200AA0F12C02BCEEC00A00
:102A000010EE101A017010EE101A090A41701449E4
:102A100091ED000A20EE200ABCEEC00A10EE101A5A
:102A2000817010EE101A090AC1700E4909880171EF
:102A3000090A41710C218171D17801F1C003C37180
:102A4000491CC8B2D070202801D30020D0700822C1
:102A500005490248FEF7A6BA540000209C00002059
:102A6000500000200C00002001534E1F144830B4C9
:102A7000144900880870000A487013480022007842
:102A800088701248CA70007810B10120087100E007
:102A90000A710F480B4C007848710F20343C887144
:102AA000E07800F1C003401CC0B2CB71E070202878
:102AB00000D3E27030BC082206490248FEF772BA21
:102AC00008000020A40000200A00002003000020CD
:102AD0000600002001534E1F1F4AFDEEC00A107071
:102AE00010EE900A51701D49F8EEE00A90FBF1F3E8
:102AF000937090FBF1F301FB130042F2107190FB15
:102B0000F1F3D37090FBF1F301FB1300642190FB10
:102B1000F1F330EE600A1371DFED110A90FBF1F36F
:102B200020EE200A01FB13005071BDEEC00A111FF8
:102B300010EE100A9071C87800F1C003401CC0B2BA
:102B4000D371C870202801D30020C870082205491D
:102B50000148FEF727BA00007400002040420F0031
:102B60000000C84201524E1F10B5264C2649A278DB
:102B700001F10C00121F0A2A11D2DFE802F0050A47
:102B8000161B20252A2F343B91ED000AF12101204C
:102B900003E091ED010AF1210220FFF79DFFA078EB
:102BA000002801D0401EA07010BD91ED020AF12155
:102BB0000320F2E790ED030AF1210720EDE790ED05
:102BC000020AF1210820E8E790ED040AF12109202A
:102BD000E3E790ED010AF1210A20DEE790ED000A1B
:102BE000F1210B20D9E794ED120AF1210D20B8EE66
:102BF000C00AD2E794ED130AF1210E20B8EEC00A04
:102C0000CBE7000000000020B003002010B5FFF764
:102C1000B1F8254C2549627801F10C000F2A14D235
:102C2000DFE802F013080D161313131B20252A2FBB
:102C300013343B0091ED000AF121012003E091EDF6
:102C4000010AF1210220FFF747FF0020607010BD4C
:102C500091ED020AF1210320F5E790ED030AF1213D
:102C60000720F0E790ED020AF1210820EBE790ED54
:102C7000040AF1210920E6E790ED010AF1210A207A
:102C8000E1E790ED000AF1210B20DCE794ED120A58
:102C9000F1210D20B8EEC00AD5E794ED130AF12119
:102CA0000E20B8EEC00ACEE700000020B0030020DE
:102CB0000CB50022274900920192086840F4803048
:102CC00008604FF4A043086800F4003001900098B9
:102CD000401C0090019810B900989842F3D1086800
:102CE000800334D5012001901A484030026842F038
:102CF000805202601848026842F44042026015485F
:102D0000083002680260026842F400420260026811
:102D100042F4A0520260031F104A1A600A6842F08F
:102D200080720A600A689201FCD50D4940F2057272
:102D30000A60016821F003010160016841F00201AD
:102D400001600168C1F381010229FAD10CBD019231
:102D50000CBD0000003802400070004008544007DD
:102D6000003C024000F8041B002120F8851B0A22C9
:102D700000F819299FED070B01764183818380EDCF
:102D80000C0B022280F83A20818780F8381080F8F6
:102D9000421070470000000000000000012080F396
:102DA0001388BFF34F8F05480168054A01F4E061BD
:102DB00011430160BFF34F8F00BFFDE70CED00E052
:102DC0000400FA05144810B502681449CB6BD21AF6
:102DD000142A20D30068C8630878421C0A700328AC
:102DE00001D300200870087848B101280DD00228CE
:102DF00011D1FFF7F9FDBDE81040FFF737BEFFF72F
:102E00002FFDBDE81040FFF763BDFFF78DFDBDE866
:102E10001040FFF7BBBD10BD600000200000002087
:102E200005490A680548436BD21A0A2A03D3096880
:102E30004163FFF799BE704760000020000000204A
:102E40002DE9F04730480168304CA26A914229D000
:102E500000682F4FA0624FF400713846FFF75EF80C
:102E60000A264FF400490025F0B125614FF4807126
:102E70003846FFF753F8DFF89C80012700B36561FF
:102E800004214046FFF74AF828B3A561E06A401CD8
:102E9000E0620A2829D80E211F48FFF79CF8216B11
:102EA00008442063BDE8F0872069401C20610228A7
:102EB000DCD949461948FFF738F8E6702581D5E78F
:102EC0006069401C60610228DAD949464046FFF734
:102ED0002CF82771D4E7A069401CA0610228D5D93D
:102EE00002214046FFF721F8D0E7E562206B40F26F
:102EF000DC51B0FBF6F06064884201D9A77100E0B4
:102F0000A5712563CEE700006000002000000020CE
:102F10000004024000000240002001400014024072
:102F20000C4900B50A680C48836BD21A142A0FD3D7
:102F30000968816309490022A1F5B870FFF7CCF94F
:102F400006490022A1F1B8005DF804EBFFF7C4B90F
:102F500000BD00006000002000000020B003002041
:102F600070B517480168174C226C891AB1F5FA7FC1
:102F700024D30068144D206401212846FEF7D9FFB0
:102F800020894FF4004608B1E07868B13146284600
:102F9000FEF7CBFF61890D4809B1217949B131466E
:102FA000BDE87040FEF7C1BF31462846FEF7BFFFBF
:102FB000F0E73146BDE87040FEF7B9BF70BD0000D4
:102FC00060000020000000200014024000000240C9
:102FD00002480168491C0160704700006000002041
:102FE000124810B5016841F4700101601048016891
:102FF00041F0010101600E4A0021083211600268AF
:103000000C4B1A400260031D0B4A1A60026822F43E
:103010008022026006480C300160FFF749FE034938
:103020004FF000608039086010BD000088ED00E0BE
:1030300000380240FFFFF6FE103000242DE9FC416D
:10304000314C0121204600F09DF8002859D0012183
:10305000204600F077F82D490878421C0A700428B1
:1030600001D30020087008784FF08063284E59146F
:10307000D8B1284D4F00012825D0022832D003288E
:103080003FD1254C2548CDE900044FF0C0632A46C6
:103090000007FEF71DFCA4F120002A46C18B02B0F8
:1030A0002046BDE8F04100F015BC19481C4C3430F6
:1030B000184DCDE90004783D2A463046FEF708FC5D
:1030C000A4F12000E9E7174C1748CDE900041648A1
:1030D0004FF020632A4639463838FEF7F9FBA4F151
:1030E0002000DAE70A48114C38300A4DCDE90004D7
:1030F000303D2A4639463046FEF7EAFBA4F120006F
:10310000CBE7BDE8FC81000000000140B0000020DA
:103110000008004088600240600200203400004047
:10312000A8010020F000002038040040180300200F
:103130000029018802D041F0800101E021F08001E6
:1031400001807047C943018270470029018802D07D
:1031500041F0010101E021F00101018070470029E7
:1031600030F8441F02D041F4004101E0C1F30E01E8
:1031700001807047002A828901D00A4300E08A4317
:103180008281704702460020138A92890B4202EA2C
:10319000010202D0002A00D001207047002A828953
:1031A00001D00A4300E08A4382817047FEB517468A
:1031B0000A4605461C4601211046089EA8470020E5
:1031C000ADF80040ADF80200ADF808000196694680
:1031D000384600F0A9F801213846FFF7A9FF202161
:1031E000384600F099F8012211463846FFF7D6FF1D
:1031F00001213846FFF7A9FFFEBD08B58DF8000094
:103200008DF801108DF8022001208DF8030068462A
:10321000FFF728F908BD000030B5028C22F001024A
:103220000284028C8388048B22F0020224F073054E
:103230000C882C438D8915434A882A430C4DA8429B
:1032400002D00C4DA8420DD122F00805CA8923F402
:1032500040732A4322F004058A882A430D8A1D43BD
:103260004B8A2B438380048389684163028430BD89
:103270000000014000040140028B22F008020A43D2
:103280000283704770B5028C22F010020284028C17
:103290008388048B0D8824F4E6464FF6FF7404EA15
:1032A000052535438E8922F0200204EA06161643CE
:1032B0004A8804EA02123243104EB04202D0104E45
:1032C000B04215D122F08006CA8923F4406304EA93
:1032D0000212324322F040068A8804EA0212324384
:1032E0000E8A04EA86061E434B8A04EA83033343AC
:1032F0008380058389688163028470BD000001407A
:1033000000040140028B4FF6FF7322F4006203EACF
:103310000121114301837047828822F0700282806C
:1033200082880A438280704730B50288164C174D58
:10333000A0420DD0A8420BD0B0F1804F08D0144B62
:10334000984205D0134B984202D0134B984203D1B8
:1033500022F070034A881A43104B984206D0104B53
:10336000984203D022F440730A891A4302804A68C3
:10337000C2620A880285A04201D0A84201D1897A9E
:1033800001860121818230BD00000140000401401E
:103390000004004000080040000C00400010004005
:1033A0000014004070B5104C40F2255529462046C7
:1033B00000F032F948B10D492046FEF7FBFD2946E1
:1033C0002046BDE8704000F08BB840F22441204612
:1033D00000F022F9002806D02088A088BDE87040BF
:1033E0000248FDF723BC70BD00500040880100205A
:1033F00070B5114C40F225552946204600F00CF9D5
:1034000048B10E492046FEF7D5FD29462046BDE8C5
:10341000704000F065B840F22441204600F0FCF80E
:10342000002808D020880448001D0088BDE87040AE
:103430000248FDF7FBBB70BD004400404002002085
:1034400070B5114C40F225552946204600F0E4F8AD
:1034500048B10E492046FEF7ADFD29462046BDE89D
:10346000704000F03DB840F22441204600F0D4F80E
:10347000002808D020880448001D0088BDE870405E
:103480000248FDF7D3BB70BD00480040D0000020CB
:1034900070B5114C40F225552946204600F0BCF885
:1034A00048B10E492046FEF785FD29462046BDE875
:1034B000704000F015B840F22441204600F0ACF80E
:1034C000002808D020880448001D0088BDE870400E
:1034D0000248FDF7ABBB70BD00140140F8020020AC
:1034E0000A0A01219140C94301807047002981895E
:1034F00002D041F4005101E021F400518181704774
:1035000038B5032000900823294A0721012000F044
:1035100063F800220321262000F036F94FF4E1344D
:103520002346244A4FF40031234800F003F90B20CE
:1035300000904FF40063214A0721022000F04CF86C
:1035400000220321272000F01FF923461C4A4FF4D4
:103550008021194800F0EEF8022008210090042391
:10356000184A084600F038F800220321352000F000
:103570000BF92346144A4FF480110F4800F0DAF893
:10358000092000904FF40073104A0821402000F0F9
:1035900023F800220321472000F0F6F801B023466B
:1035A000BDE830400A4A20210A4800F0C3B80000B4
:1035B0000000024000440040692500080004024069
:1035C00000480040000C024000500040001802403B
:1035D00000140140812500082DE9FC410E461C46DF
:1035E00015460121089FFEF7B3FF324639462846AB
:1035F000FEF784FC02218DF804108DF805100020E0
:103600008DF8060001208DF80700009469462846D1
:10361000FEF738FCBDE8FC8170B501F01F050126FE
:103620000024C1F3421306FA05F2012B0FD0022B3E
:103630000FD0838A4FEA11210088134206FA01F65F
:1036400000EA060001D000B10124204670BD838944
:10365000F0E7038AEEE710B5C1F3421301F01F044F
:103660000121A140012B07D0022B07D01430002AE2
:10367000026805D00A4304E00C30F8E71030F6E7A2
:103680008A43026010BD00007FB50446008A0D46E3
:10369000C98820F4405001432182A08941F20C6185
:1036A0008843A9882A8911436A8902431143A18169
:1036B000A08A20F44071A8890843A0826846FEF7DA
:1036C00077FF1A48844202D01948844201D10398F6
:1036D00000E00298A189090400EBC00101EB001091
:1036E000296801D5490000E08900B0FBF1F06422AF
:1036F000B0FBF2F109010B096FF018056B4300EB09
:103700008300A3891D044FF0320306D503EBC000EC
:10371000B0FBF2F000F0070005E003EB0010B0FB97
:10372000F2F000F00F00084320817FBD001001403F
:10373000001401407FB516460A4605461C46012185
:103740001046A8470020ADF80800ADF80400042199
:10375000ADF80600ADF80A10ADF80C00009469460B
:103760003046FFF791FF012240F225513046FFF726
:1037700072FF012240F224413046FFF76CFF012125
:103780003046FFF7B3FE7FBD08B58DF800008DF819
:1037900001108DF8022001208DF803006846FEF725
:1037A00061FE08BD8088C0F30800704702E008C8C9
:1037B000121F08C1002AFAD170477047002001E0AB
:1037C00001C1121F002AFBD170474FF6FF7101EAB9
:1037D00040000022034611464240491C0011C9B274
:1037E0000329F9D302F00F0040EA031080B27047BA
:1037F0001FB56846FEF7DCFE0D490098B0FBF1F0FE
:103800000C49086001984FF47A71B0FBF1F0401E4A
:10381000B0F1807F0AD24FF0E0214861064AF020E3
:1038200082F8140D00208861072008611FBD000088
:1038300040420F005C0000200FE000E030B504467D
:10384000FEF72EFD054604EB4400C0EBC414FEF762
:1038500027FD401BB0EBC40FF9D330BD70B5064651
:1038600000200D46044606E0325D0146104600F099
:10387000A3F8641CE4B2AC42F6D370BDFDF78AF93C
:103880004FF48060FEF720FEFFF7B2FFFEF722FA4A
:10389000FEF764F8FCF798FFFDF7B4FBFFF730FE86
:1038A000FEF7F6FCFEF724FE40F6B830FFF7C6FF41
:1038B0004FF47A710420FEF7B4FCFFF7C1FAFFF76A
:1038C000AFFAFFF72DFBFFF77DFAFFF749FBFEF795
:1038D00005FEF2E770B515460446B1F5006F02D358
:1038E00040F2FF7000E00846FFF76FFF010401D5CA
:1038F000342100E01A212160410401D5342100E087
:103900001A216160810401D5342100E01A21A160EF
:10391000C10401D5342100E01A21E160010501D57F
:10392000342100E01A212161410501D5342100E054
:103930001A216161810501D5342100E01A21A161BC
:10394000C10501D5342100E01A21E161010601D54C
:10395000342100E01A212162410601D5342100E022
:103960001A216162810601D5342100E01A21A16289
:10397000C10601D5342100E01A21E162010701D519
:10398000342100E01A212163410701D5342100E0F0
:103990001A216163810701D5342100E01A21A16356
:1039A000C00701D0342000E01A20E0632846BDE8BB
:1039B00070400121FDF762BE484000210722030646
:1039C00002D582EA400000E04000491CC9B2C0B202
:1039D0000829F4D370470000F839000800000020DF
:1039E000CC000000AC370008C43A0008CC0000202E
:1039F0001C070000BC3700080000000000000000A9
:103A000000000000000000000000000000000000B6
:103A100000000000EF1D953D5932C7BB0B604A39CD
:103A20000000000000000000000000000000000096
:103A30000000000000000000000000000000000086
:103A40000000000000000000000000000000000076
:103A50000000000000000000000000000000000066
:103A60000000000078563412000000000000000042
:103A70000000000000000000000000000000000046
:103A80000000000000000000000000000000000036
:103A90000000000000000000000000000000000026
:103AA0000000000000000000000000000000000016
:103AB00000000000000000000102030401020304F2
:043AC00006070809E4
:040000050800018965
:00000001FF
